:1000000000308A00802A0000831A0A28A300030E09
:10001000A4000F288312A300030EA400A414A30EAF
:100020000408A5000C08A6000D08A70083128B1E6B
:100030001B280B191C280900A0308100061A222851
:1000400000302328013094001608960A1408031D76
:100050004F2801301802031D4F280E3016020318D6
:1000600035280530160203183828960195014F28C7
:100070000A301602031C46280830150203184628C9
:100080001508950A0314970C96014F28083015029D
:1000900003184F281508950A0310970C960108308D
:1000A0001502031D572809309500170899001408F8
:1000B0009800861A5D2800305E2801309A001A08E0
:1000C000031D972801301D02031D97288B138530CF
:1000D0008C008C0B692801309F0009301F02031827
:1000E0008528861A75280030762801309A001A086B
:1000F000031D7C2803107D2803149B0C85308C0085
:100100008C0B80281F089F0A6D28861A89280030CA
:100110008A2801309A0001301A02031D95281B0815
:100120009E0030309E021E088F0001309C001A088D
:100130009D000B112508840026088C0027088D00DF
:10014000240E83008312230EA418831609002B08A3
:100150000319B72801308D008C018C0BAD288D0B55
:10016000AC284A308C008C0BB328AB0BAA28003487
:100170002908031DBD288610C12801302902031952
:10018000861485308C008C0BC328003406118B1329
:10019000A901B820280801398C0001300C02031D88
:1001A000D5280130A900B820D728A901B8202808EF
:1001B00002398C0003108C0C0C088C0001300C02EE
:1001C000031DE6280130A900B820E828A901B820BD
:1001D000280804398C008C0C8C0C3F308C050C08E2
:1001E0008C0001300C02031DF9280130A900B82051
:1001F000FB28A901B820280808398C008C0C8C0C2D
:100200008C0C1F308C050C088C0001300C02031D77
:100210000D290130A900B8200F29A901B82028080C
:1002200010398C008C0E0F308C050C088C000130BE
:100230000C02031D1F290130A900B8202129A901A2
:10024000B820280820398C008C0E8C0C07308C05C7
:100250000C088C0001300C02031D32290130A9006A
:10026000B8203429A901B820280840398C008C0E08
:100270008C0C8C0C03308C050C088C0001300C02AB
:10028000031D46290130A900B8204829A901B8203A
:10029000280880398C008C0E8C0C8C0C8C0C013056
:1002A0008C050C088C0001300C02031D5B29013009
:1002B000A900B8205D29A901B8200130A900B82003
:1002C0008B170615003486110000000000000000A6
:1002D0000000861506308C008C0B6C2986110000FE
:1002E0000000000000000000861506308C008C0B1A
:1002F000772986110000000000000000000086152C
:1003000006308C008C0B8229861100000000000052
:1003100000000000861506308C008C0B8D2986119C
:1003200000000000000000000000861506308C0070
:100330008C0B98292A08031DA32942308C008C0BB2
:100340009F290000C82901302A02031DAF2901306E
:10035000AB00A72021308C008C0BAC29C8290230BF
:100360002A02031DC12953308C008C0BB529533050
:100370008C008C0BB92910308C008C0BBD2900002F
:10038000C82903302A02031DC8290230AB00A72068
:1003900000348B13AA016321290801398C00013034
:1003A0000C02031DD7290130AA006321DA2902308B
:1003B000AA006321290802398C0003108C0C0C0858
:1003C0008C0001300C02031DE9290130AA006321D1
:1003D000EC290230AA006321290804398C008C0C16
:1003E0008C0C3F308C050C088C0001300C02031D76
:1003F000FD290130AA006321002A0230AA006321EE
:10040000290808398C008C0C8C0C8C0C1F308C0546
:100410000C088C0001300C02031D122A0130AA00C6
:100420006321152A0230AA006321290810398C00A3
:100430008C0E0F308C050C088C0001300C02031D53
:10044000252A0130AA006321282A0230AA0063214C
:10045000290820398C008C0E8C0C07308C050C0878
:100460008C0001300C02031D392A0130AA006321DF
:100470003C2A0230AA006321290840398C008C0EE6
:100480008C0C8C0C03308C050C088C0001300C0299
:10049000031D4E2A0130AA006321512A0230AA000E
:1004A0006321290880398C008C0E8C0C8C0C8C0CF0
:1004B00001308C050C088C0001300C02031D642AED
:1004C0000130AA006321672A0230AA0063210330A9
:1004D000AA0063218B17003401308E000130A9007F
:1004E000C9210F08A900C9210F088E0601300E028C
:1004F000031D7C2A02308E000E08A900C921FA2AA9
:10050000840195019601013098009C0101309D0005
:100510008B133030660008308C008C1D972A073012
:100520008101813084000008C0390F3880006400E8
:10053000813084000008C0390C0480008B1606113D
:100540000230A800FA30AB00A720A80BA22A06159B
:100550008B171C08031DF02A09301502031DEF2A12
:1005600095012108031DBD2A01301902031DBD2A72
:100570001908A2000130A100EF2A01302102031C5A
:10058000D22A053021020318D22A013021028C0020
:1005900010300C078400190880001908A2062108F1
:1005A000A10AEF2A05302102031DEE2A01302202A2
:1005B000031DDC2A0230A20022081902031DEC2AC6
:1005C0001008A800C6201108A800C6201208A8001C
:1005D000C6201308A800C620A101EF2AA101FF2A06
:1005E00001301C02031DFF2AA00132302002031833
:1005F000FD2A6C2A2008A00AF52A9C018B17A92A3B
:100600006300FF3FFF3FFF3FFF3FFF3FFF3FFF3FD5
:10061000FF3FFF3FFF3FFF3FFF3FFF3FFF3FFF3FEA
:10062000FF3FFF3FFF3FFF3FFF3FFF3FFF3FFF3FDA
:10063000FF3FFF3FFF3FFF3FFF3FFF3FFF3FFF3FCA
:10064000FF3FFF3FFF3FFF3FFF3FFF3FFF3FFF3FBA
:10065000FF3FFF3FFF3FFF3FFF3FFF3FFF3FFF3FAA
:10066000FF3FFF3FFF3FFF3FFF3FFF3FFF3FFF3F9A
:10067000FF3FFF3FFF3FFF3FFF3FFF3FFF3FFF3F8A
:10068000FF3FFF3FFF3FFF3FFF3FFF3FFF3FFF3F7A
:10069000FF3FFF3FFF3FFF3FFF3FFF3FFF3FFF3F6A
:1006A000FF3FFF3FFF3FFF3FFF3FFF3FFF3FFF3F5A
:1006B000FF3FFF3FFF3FFF3FFF3FFF3FFF3FFF3F4A
:1006C000FF3FFF3FFF3FFF3FFF3FFF3FFF3FFF3F3A
:1006D000FF3FFF3FFF3FFF3FFF3FFF3FFF3FFF3F2A
:1006E000FF3FFF3FFF3FFF3FFF3FFF3FFF3FFF3F1A
:1006F000FF3FFF3FFF3FFF3FFF3FFF3FFF3FFF3F0A
:10070000FF3FFF3FFF3FFF3FFF3FFF3FFF3FFF3FF9
:10071000FF3FFF3FFF3FFF3FFF3FFF3FFF3FFF3FE9
:10072000FF3FFF3FFF3FFF3FFF3FFF3FFF3FFF3FD9
:10073000FF3FFF3FFF3FFF3FFF3FFF3FFF3FFF3FC9
:10074000FF3FFF3FFF3FFF3FFF3FFF3FFF3FFF3FB9
:10075000FF3FFF3FFF3FFF3FFF3FFF3FFF3FFF3FA9
:10076000FF3FFF3FFF3FFF3FFF3FFF3FFF3FFF3F99
:10077000FF3FFF3FFF3FFF3FFF3FFF3FFF3FFF3F89
:10078000FF3FFF3FFF3FFF3FFF3FFF3FFF3FFF3F79
:10079000FF3FFF3FFF3FFF3FFF3FFF3FFF3FFF3F69
:1007A000FF3FFF3FFF3FFF3FFF3FFF3FFF3FFF3F59
:1007B000FF3FFF3FFF3FFF3FFF3FFF3FFF3FFF3F49
:1007C000FF3FFF3FFF3FFF3FFF3FFF3FFF3FFF3F39
:1007D000FF3FFF3FFF3FFF3FFF3FFF3FFF3FFF3F29
:1007E000FF3FFF3FFF3FFF3FFF3FFF3FFF3FFF3F19
:1007F000FF3FFF3FFF3FFF3FFF3FFF3FFF3FFF3F09
:00000001FF
